:100000000450000087329A0227BF0221B20000008C
:10001000000002001E0000000000000000000000C0
:10002000000002011A853F8C85408AC0E0C0D0C024
:10003000F0C082C083C000C001C002C003C004C0C1
:1000400005C006C007E53E2408F8E6602BE53E241F
:1000500010F8A681E53E75F021A42405F582E4346C
:10006000F8F583788CE58104C398F9942240030263
:1000700011DCE6F008A3D9FA7408253EF8053E081D
:10008000E65480700CE53EB407F37808753E0080B6
:10009000EFE53E2410F88681E53E75F021A42405A5
:1000A000F582E434F8F583788CE58104C398F9E0AF
:1000B000F608A3D9FAD007D006D005D004D003D0D3
:1000C00002D001D000D083D082D0F0D0D0D0E032A6
:1000D00030014D30B44810004590FF08E05420F83E
:1000E00090FF48E05420F990FF10E05420FA90FF70
:1000F00050E05420FB7400F58274F8F583E0C8F0FA
:100100006860027E04A3E0C9F06960027E04A3E097
:10011000CAF06A60027E04A3E0CBF06B60027E044A
:1001200022C0E0C0D0C0F0C082C083C000C001C007
:1001300002C003C004C005C006C0077415F5827470
:10014000F9F583E060237466F58274F9F583E014B1
:10015000F0701674FFF0741CF58274F9F583E0609A
:100160000414F07004C29080FC90FF937481F0E559
:100170008194FD40030211DC85418D85428B74B270
:10018000F58274FAF583E0B4011BC082C08390FF4E
:100190004AE030E72C90FF4EE030E725D083D08254
:1001A0007402F08020B4021DC082C08390FF7AE008
:1001B00030E70512284E8009D083D0827403F08086
:1001C00004D083D082A3E0B4011BC082C08390FF1F
:1001D00052E030E72C90FF56E030E725D083D08204
:1001E0007402F08025B40222C082C08390FF7AE0BE
:1001F00030E70512284E8009D083D0827403F08046
:1002000009D083D08280030202907416F58274F9BB
:10021000F583E02004F12002033001EB7419F5822C
:1002200074F9F583E014FCF0A3E0FDA3E0FE6404A0
:10023000700FEC70627E011200C97C0A7DFA020226
:10024000611200C9EE6404601DEC704B7C0AED1471
:10025000FD7015EE640260077E027D320202617E4F
:10026000017DFA0202617C0A7419F58274F9F58342
:10027000ECF0A3EDF0A3EEF014601820E10F2001E4
:1002800006D2B1C2B08010C2B1D2B0800AC2B1C22F
:10029000B08004D2B0D2B1781979097A07E7700436
:1002A000A600800BE6600816E67004E74480F708B5
:1002B00009DAEAE53D601314F53D700EE53E2408C9
:1002C000F87600121157D28CD28DD007D006D00507
:1002D000D004D003D002D001D000D083D082D0F09F
:1002E000D0D0D0E03290FF04E090FAB9F090FF0651
:1002F000E0FCA3E0FAECFFEAFEEFC39408EE940101
:10030000500280047E017F088E3B8F3C90FF02E00C
:10031000FCA3E0FAECFFEA90FABDF0EFA3F0121CA8
:10032000E0E4F54DE54DC39402500F121CC1E412F8
:100330001AE8054D04121CB280EA121CE090FF007E
:10034000E0FF546024C070030208F32440600302FD
:100350000F6E90FAB9E0FE540FF54DEE30E703D37F
:100360008001C3920A90FF01E0121BFC0384000489
:100370005701056A0306310506730607D508081DEF
:100380000908790A08B90B00000F6EE53520E7036C
:10039000020F6E90FABDE07002A3E06003020F6EE0
:1003A000E53C6402453B6003020F6EEF541F14608E
:1003B0002B14604724026003020F6EEE6003020FED
:1003C0006E121CC17401121AE87867E630E0081258
:1003D0001CC17402121AE87F0202326EE53520E178
:1003E0000990FAB9E06003020F6E90FAB9E0D39475
:1003F000014003020F6E7F0202326EE53520E10EEE
:1004000090FAB9E0FF600764806003020F6E120F7C
:10041000FA4003020F6EE54D7019300A0B90FF8011
:10042000121CBE121AE8802490FF82121CBE121AFF
:10043000E88019154D300A0B121D55121CBC121AFA
:10044000E88009121D63121CBC121AE8121CC112AA
:100450001AA260057401121AE87F0202326EE535B5
:1004600030E703020F6EE53C453B6003020F6E125E
:100470001D7914602D14605924026003020F6E90E0
:10048000FABDE07004A3E064016003020F6E90FA0D
:10049000B9E06003020F6E7867E654FEF6E4FF02EF
:1004A000326EE53520E10620E003020F6EE53530BF
:1004B000E00990FAB9E06003020F6EE53530E10C17
:1004C00090FAB9E0D394014003020F6EE4FF0232C8
:1004D0006E90FABDE07002A3E06003020F6E120F8F
:1004E000FA4003020F6EE53520E10620E003020F1B
:1004F0006EE53530E007E54D6003020F6EE54D70A7
:100500000F90FF82E054F7F090FF80E054F7F02264
:10051000E54D24FE602024FB603424067035300A4B
:100520000CA20AE433FD7F03122E798026E4FD7FBE
:1005300003122E79801D300A0CA20AE433FD7F04D9
:10054000122E79800EE4FD7F04122E7980057F87BC
:100550001231EF154D300A0B121D55F583E054F79B
:10056000F08009121D63F583E054F7F0E4FF0232D6
:100570006EE53530E703020F6EE53C453B60030254
:100580000F6E121D7914602D146055240260030251
:100590000F6E90FABDE07004A3E064016003020FE7
:1005A0006E90FAB9E06003020F6E7867E64401F6D8
:1005B000E4FF02326EE53520E10620E003020F6E13
:1005C000E53530E007E54D6003020F6EE53530E1BB
:1005D0000AE54DD394014003020F6EE4FF02326E30
:1005E00090FABDE07002A3E06003020F6E90FAB9CA
:1005F000E0FF12323F4003020F6EE53520E1062096
:10060000E003020F6EE54D7009300A03021E14026A
:100610001DDFE53520E103020F6E154D300A0B1288
:100620001D55F583E04408F08009121D63F583E051
:100630004408F0E4FF02326EE53530E703020F6E46
:10064000E53C453B6003020F6E90FAB9E06003029F
:100650000F6E121D796003020F6EE53530E1030263
:100660000F6E90FABEE090FFFFF0E06005433501A9
:1006700080035335FEE4FF02326EE53520E70302C6
:100680000F6EE53C453B7003020F6E121D7960034F
:10069000020F6E90FABDE0FCA3E0FDEC24FE603A90
:1006A00014607524026003020F6EED6003020F6E8A
:1006B000121CE0121E0D7D03120FB56003020F6EB7
:1006C000120F7290FAB6E0FDA3121D2B120FD1503B
:1006D000028004AE3BAF3C021002121CE090F916FF
:1006E000E030E40D121E0D7D14120FB56010020FE4
:1006F0006E121E0D7D041210096003020F6E120FA0
:100700007290FAB6E0FDA3121D2B120FD150028099
:1007100004AE3BAF3C021002121E0D7D0512100903
:100720006003020F6E7B017AFA79B6121D287D01F3
:1007300012269890FAB7E475F003121B1C90FABECB
:10074000E090FAB5F0E4F54C90FAB5E0FFE54CC363
:100750009F5024121D22121014FFFD90FAB7E48D51
:10076000F0121B1C90FAB6E0C39FF0D39400500324
:10077000020F6E054C80D1121D2212101424FEFFB0
:1007800090FAB6F0FDA3E475F002121B1C7AF97919
:10079000727B018B368A378938E92402F9E43AFA08
:1007A000121D281226988F4C054C054C121CC1E5D1
:1007B0004C121AE8121CC19000017403121AFAAF0D
:1007C0004C7E00C3EF953CEE953B50028004AE3B5F
:1007D000AF3C8E398F3A022CD8020F6EE53520E7F8
:1007E00003020F6EE53C6401453B6003020F6E900F
:1007F000FAB9E06003020F6E90FABDE07002A3E068
:100800006003020F6E121D796003020F6EE5352042
:10081000E00620E103020F6E75360075370075386B
:1008200032020FF1E53530E703020F6EE53C453B40
:100830006003020F6E90FAB9E06003020F6ED3906E
:10084000FABEE0940190FABDE094004003020F6EFE
:10085000121D796003020F6EE53520E00620E103EA
:10086000020F6E90FABEE0F532E5327008433501B2
:100870005335FD80065335FE433502E4FF02326EE8
:10088000E53520E703020F6EE53C6401453B60035C
:10089000020F6E90FAB9E06003020F6E90FABDE0AD
:1008A0007002A3E06003020F6E121D796401600301
:1008B000020F6EE53520E103020F6E7F0102326EFA
:1008C000E53530E703020F6EE53C453B6003020F60
:1008D0006ED390FABEE0940090FABDE0940040031D
:1008E000020F6E121D7964016003020F6EE5352060
:1008F000E103020F6EE4FF02326E90FF01121E242C
:10090000EF121AE890FAB9121E24900001EF121AA1
:10091000FA900002E4121AFA7403121CB290FABDA3
:10092000E0FFA3E0853882853783CFF0A3EFF09016
:10093000FF01E0121BFC097B02099D0409BF0509A8
:10094000EB060A09070A27080A45090A630B0B1870
:10095000800DB7810DE8820B5F830BA8840BC785E0
:100960000C0C860C57870CE8880D73890A81920A53
:1009700081930DA0B00E9BC00EC7C10ED8C200005F
:100980000F5DE53520E7057F050231A9121D716075
:1009900003047009EFFD7C007F0702115EE4FD7F18
:1009A00007022FB4E53520E7057F050231A9121DA6
:1009B000716003047009EFFD7C007F0C02115EE49E
:1009C000FD7F07022FB4E53530E703020F71121ED9
:1009D000425006E53C453B70057F020231A990FA82
:1009E000B9E024FE24FD5002800302322C7F07026E
:1009F00031A9E53530E703020F71121D7160030460
:100A00007009EFFD7C007F0802115E7F070231A9AB
:100A1000E53530E703020F71121D716003047009A0
:100A2000EFFD7C007F0902115E7F070231A9E535E9
:100A300030E703020F71121D716003047009EFFDAE
:100A40007C007F0A02115E7F070231A9E53530E79D
:100A500003020F71121D716003047009EFFD7C0029
:100A60007F0B02115E7F070231A9E53530E70302F3
:100A70000F71121D716003047009EFFD7C007F0E81
:100A800002115E7F070231A9E53530E756121D7964
:100A9000704A90FF02E0F54CE54CB48205754C615C
:100AA0008012E54CB48305754C628008E54CC45453
:100AB000F004F54C121C22121E3B1225FA121D895D
:100AC000121ABB600512327A800685333985343AB2
:100AD0007536017537F9753875022CD8E4FD7F0538
:100AE000022FB4121D7960057F050231A9121E4242
:100AF00040057F030231A990FF02E0F54CE54CB4BC
:100B00008205754C618012E54CB48305754C62809A
:100B100008E54CC454F004F54C121C2202322C128D
:100B20001E4C122AC7121D33E0547FF0000000E073
:100B300090FABAF07868121BD8900002121ABB30F3
:100B4000E7F2900002E4121AFA90FABAE04480FF49
:100B5000F0787CE6FC08E68C83121D3BEFF0123245
:100B600084E4FF0231A990FAB9E06401701F90FAA1
:100B7000BDE0FF7E007006A3E0F590802DC2AFEFD0
:100B8000F4529090FABEE04290D2AF801D90FABD30
:100B9000E0FF7E007006A3E0F5B0800EC2AFEFF478
:100BA00052B090FABEE042B0D2AFE4FF0231A912D7
:100BB0001CE090FAB9E0B4010A121CC1E590121AC7
:100BC000E88008121CC1E5B0121AE8020FF190FA91
:100BD000B9E0FF2413121CF120E133121D80EF2431
:100BE000FC601804702890FABAE0600990FFA4E055
:100BF0004410F08019121E56F0801390FABAE0608B
:100C00000990FFB4E04410F08004121E5DF0E4FF90
:100C10000231A990FAB9E0FF2413121CF120E13946
:100C2000121D80EF24FC601B04702E90FABAE06065
:100C30000990FFA4E04420F0801F90FFA4E054DF5F
:100C4000F0801690FABAE0600990FFB4E04420F01A
:100C5000800790FFB4E054DFF0E4FF0231A9121DD9
:100C600080121D71604D046003020CE390FABAE03B
:100C7000600F90FFA4121CEA30E16F121E2C020CD0
:100C8000E390FFA4E054FB121CEDFE30E15C30E287
:100C90001130B405121E2C805190FFA4E054FDF0D9
:100CA0008048309505121E2C804090FFA4E054FD32
:100CB000F0803790FABAE0601290FFB4121CEA306C
:100CC000E12890FFB4E04402F0801F90FFB4E054AC
:100CD000FB121CED30E11330930990FFB4E04402A5
:100CE000F0800790FFB4E054FDF0E4FF0231A91258
:100CF0001D8090FAB9E024FC604004707890FABA44
:100D0000E0601D90FFA2E04440F0A3E0FF30E76503
:100D1000D203A3E054DFF090FFA3EF547FF080559F
:100D200030030E90FFA3E04480F0C203A3E0442010
:100D3000F090FFA2E054BFF0803B90FABAE0601D53
:100D400090FFB2E04440F0A3E0FF30E728D204A3D4
:100D5000E054DFF090FFB3EF547FF0801830040EC2
:100D600090FFB3E04480F0C204A3E04420F090FF81
:100D7000B2E054BFF0E4FF0231A9121CE090FAB9CE
:100D8000E024FC600F04701690FFA6E0121CC11254
:100D90001AE8800A90FFB6E0121CC1121AE87539F1
:100DA00000753A01022CD890F9157401F090F91CE5
:100DB0007419F090F96674FFF0E4FF0231A9E4FFC2
:100DC0001231A9121DE77F0312126190F916E0306B
:100DD000E40890FF937480F0801090FFFCE0547F53
:100DE000F07FFF7E001230D3C290C2AF0080FDE4DE
:100DF000F54EF54F90FABF743EF0A3E4F090FAB7C9
:100E0000F0A37415F0E0543FFFC374409F90FABC08
:100E1000F0D39400E4943E400890FAC0E090FABC0D
:100E2000F0120F98E53145307073121CFA90FABF3A
:100E3000121E066027D3EF9440EE9400400890FA0B
:100E4000BC7440F0800890FAC0E090FABCF0120F39
:100E500098E53145307046121CFA80D1754C0290ED
:100E6000FABFE4F0A304F090FAB7E4F0A3740FF033
:100E70007B007A00794C90FAC0E0F54A7D0F7C0047
:100E80001229607530008F317B007A00794CE4F5CF
:100E90002DF52E7D01122698E4F530F531AF3102A3
:100EA00031A9121D8030E710E0540F90F967F0D39C
:100EB00094004015C295801190FABAE0540F90F951
:100EC00065F0D394004002C294E4FF0231A9121EDF
:100ED0004CBF0104D2938002C293E4FF0231A912F5
:100EE0001D80540314600A14600F146008240370FA
:100EF0002BD2918027C2918023121E56120FC06000
:100F000004D291801790FFA4E04410120FC0FFBFDD
:100F1000A004C2918002D291121E56F090FABAE05B
:100F2000540CFF1313543F14600A14600F1460082C
:100F30002403702BD2928027C2928023121E5D124E
:100F40000FE06004D292801790FFB4E04410120FBB
:100F5000E0FFBFA004C2928002D292121E5DF0E4B4
:100F6000FF0231A9E53530E707E4FD7F05022FB424
:100F70007F050231A912327A227B017AFA79B69082
:100F8000FAB7E0F52DA3E0F52E7D0112269890FA30
:100F9000B7E475F003121B1CAB36AA37A93822AA96
:100FA0004EA94F7BFF90FAB7E0FCA3E0FD90FABC9E
:100FB000E0F54A1229607530008F31221223617EDC
:100FC000008E308F31EF22F07F0112126190FFA668
:100FD000E090FABBF054A0221226988F4C7E00C3FA
:100FE000EF953CEE953B22F07F0112126190FFB627
:100FF000E090FABBF054A022753900753A01022C3A
:10100000D890FAB9E0FF02323F8E398F3A022CD8DD
:101010001223617E008E308F31EF227D01122698DF
:1010200090FAB4E022EF90F804F022C0A8C2AFEE2C
:10103000600AC0057D7FDDFEDEFAD005EFC39415A2
:101040005003D0A822137003D0A822FFD507FDD0EB
:10105000A822C000C001C002C004C005E53E2408AB
:10106000F8860553057F7CFF1210C07F007E00E5E7
:10107000436046FC90F91DE0547F6D700FC083C043
:1010800082A3E0FEA3E0FFA315438007A3A3A3DC94
:10109000E68026DC06D082D083801EE0F8A3E0F94B
:1010A000A3E0FAD082D083E8F0A3E9F0A3EAF0A3AA
:1010B000C083C082A3A3A380DA121157D005D00445
:1010C000D002D001D0002285A84475A888EC700217
:1010D0007C3F8C3D22E53E2408F876001211AE805C
:1010E000FBC000C001C002C004C0067CFF1210C0DB
:1010F000E5436042FE90F91DE0547F6F700BC083A2
:10110000C082A3A3A315438007A3A3A3DEEA80267E
:10111000DE06D082D08380D8E0F8A3E0F9A3E0FA1D
:10112000D082D083E8F0A3E9F0A3EAF0A3C083C0A3
:1011300082A3A3A380DA7808087918097C01E65411
:101140007F6F700676007700800608090CBC08EEF9
:10115000121157D006D004D002D001D00022753D24
:10116000008544A822C0F0C082C083C3E54324E8C0
:1011700050051211AE80F4EF6031903111E493C349
:101180009F402FC0047CFF1210C0D004430780E5AD
:101190004375F003A4241DF582E434F9F583EFF0E0
:1011A000ECA3F0EDA3F00543121157D083D082D009
:1011B000F0220211DCC0047C20D28CD28DD504FD3B
:1011C000D0042275A80075880075B80075F0007508
:1011D000D000E4F890F804F0900000F608B800FBA6
:1011E000020000C2AFE490FF48F090FF50F090FF83
:1011F00008F090FF10F090FF80F0A3A3F0D2B1C2EE
:10120000B07EFF7FFF1210247EFF7FFF1210247E2E
:10121000FF7FFF121024D2B0D2B17EFF7FFF1210E9
:10122000247EFF7FFF1210247EFF7FFF1210248098
:10123000CCC3EE940250047E037FE8EFF4FFEEF49B
:10124000FE0FBF00010E8F428E4122C3EF94BCEE11
:10125000940250047E077FD0EFF4FFEEF4FE0FBF40
:1012600000010E8F408E3F22EF700122C000C0A807
:10127000C2AFE53E2418F8A607E53E2408F8C65498
:101280007FF6D0A8E630E703D000221211AE80F43A
:10129000C0007F01EF2408F8E660090FBF08F512CF
:1012A00011AE80EED00022C0F0C082C083C000C06A
:1012B00006C004ED2410F8769AED75F021A42405FB
:1012C000F582E434F8F583C082C083A3A3E4780DEB
:1012D000F0A3D8FCEF547F75F002A424F3F582E567
:1012E000F03430F583E493FE740193FCD083D08214
:1012F000ECF0A3EEF0ED2408F8EF4480F6D004D033
:1013000006D000D083D082D0F022753E0075430015
:101310007A0879187808760077000809DAF890F8E2
:1013200004E0FC903111E493C39C5005E490F80470
:10133000F078087480447FF674014410F58975B81C
:1013400000D2ABD2A92275818BD28ED28CD2AFE5DE
:10135000436036FF90F91DE05480602878087908D2
:10136000E0547FFA7B00E6547FB502027BFF08D988
:10137000F5EB7010EAF0C007121289AD07AF021248
:1013800012A0D007A3A3A3DFCE1211AE80C18F2479
:10139000122AC71222B5A3A3E0A330E728787E1251
:1013A0002299E04401F01222FA12229DE020E0F698
:1013B0001223507402F01222DAE0A330E507122360
:1013C00050E04401F07880E6FE08E6FF8E832408B2
:1013D0001222A1E0FD1223398A83240A1222A1EDF0
:1013E000F012230624071222A1E0FF12235A240937
:1013F0001222A1EFF090F916E030E420081222B793
:10140000C083C082A3E025E0FF0582D58202158358
:101410001582E033D082D083F0A3EFF01222B5E042
:10142000FCA3E0FDECFF1223398A8324081222A1D9
:10143000EFF0ED12235A24071222A1EDF01222A997
:10144000E030E60A12234124091222A1E4F012221C
:10145000A9E0FF30E71B12231E24091222A1E0603D
:10146000091222A9EF4402F080071222A9EF54FDCD
:10147000F0787E1222B7A3A3E0FF5307C708E6FC6B
:1014800008E6FD1222E0A3E030E3128D828C83E5B2
:101490008224051222A1E09032519342075307FBA8
:1014A00012231E24061222A1E060034307045307FF
:1014B000FC788012232924041222A1E0420743076A
:1014C00080122339F5828A83A3A3EFF012235A24D2
:1014D000041222A1E0FF8D828C83A3A3E0FCA3E091
:1014E000FD30E1055307DF8003430720EC30E405BE
:1014F0005307EF80034307101222A9E0FE54036054
:10150000735307DFEE30E16912231E24091222A172
:10151000E0121BFC152C0015600115650315600514
:1015200015650715600915650B15600D15650F002C
:1015300000156DE5246403702190F916E030E20D8A
:1015400030B405430702802C5307FD8027309505F2
:10155000430702801F5307FD801A3093054307029B
:1015600080125307FD800D43070280085307FD805A
:10157000035307FD12232724041222A1EFF08D82CA
:101580008C83A3A3A3E0FF1222A9E0FE54037003FF
:10159000021660EE20E10302165D081223202409E2
:1015A0001222A1E0121BFC15BF0015F50115F50371
:1015B000162905162907160F09160F0B16430D16C7
:1015C000430F00001660E5246403702390F916E0D1
:1015D00030E20F30B10653077F02166043078002E6
:1015E000166030940553077F807D430780807830F4
:1015F000920553077F8070430780806BE524B40316
:101600000990FF9EE054EFF0800790FF9EE054DFCA
:10161000F053077F8051E524B4030990FF9EE04416
:1016200010F0800790FF9EE04420F053077F803742
:10163000E524B4030990FF9EE054EFF0800790FF8B
:101640009EE054DFF0430780801DE524B403099039
:10165000FF9EE04410F0800790FF9EE04420F0439E
:101660000780800353077F1222DAE0FCA3E0FD30FD
:10167000E00543072080035307DFEC30E305430711
:101680004080035307BFEC30E0054307108003534D
:1016900007EFED30E40543070880035307F7ED300B
:1016A000E50543070480035307FBED30E6054307D8
:1016B0000180035307FEED30E70543070280035323
:1016C00007FD787E1222DCA3EFF01232847F002225
:1016D00090FFFA7408F0A37416F090FFF97402F00A
:1016E0007B017AFA79CFE4FD12236190FACFE47599
:1016F000F003121B1C121992E52330E702D2027B81
:10170000007A00792490FACFE0F52DA3E0F52E7D44
:101710000112269890FACFE4F0A3740BF07B007AC4
:10172000007923752D00F52E7D01122698E52324DE
:101730008090FFF8F0E5236407601EE523640660EF
:1017400018E52364146012E5236441600CE523640A
:101750001A7046E52464027040E523B40716D2945B
:10176000D295D292D29390F916E04402F0A3E044CD
:1017700002F0801EE523B4411290F916E04406F011
:10178000A3E04406F0D2B1D2B4800790F916E04449
:1017900001F090F917E04401F0E5236442600CE5A4
:1017A0002364436006E5236444702E90F916E0FF3D
:1017B000E523B444047E4080027E00EE24804F90F6
:1017C000F916F0A3E0FFE523B444047E4080027ED6
:1017D00000EE24804F90F917F090FACFE4F0A37454
:1017E0000DF012199290FFF5E523F0E4F535F5338D
:1017F000F534F532121E34121CE0121E3B90F96AC9
:10180000121BF390F96F121BF390FFFFE4F090FFAF
:1018100083E0E4F090FF817480F0A37484F090FF83
:1018200080F0E4F523E523121D57F583E4F0E5236A
:10183000121D65F583E4F00523E523B407E7787A04
:1018400076FE0876F090320AE493FF7878F6FDADE4
:1018500007903217E493FF08F6FFED540FFD121DB9
:10186000477484F0ED75F008A42447F582E434FF52
:10187000F583EFF0C374F09F787BF674FE94001844
:10188000121CD8CEC313CE13D8F9FFED121DA8EF4A
:10189000F0ED121DCEE4F523E52390320493FF789A
:1018A00078F6FDE52325E0240BF582E43432F58358
:1018B000E49308F6ED30E75318E6540FF9121D478C
:1018C000121DB62447F582E434FF121CC8CEC313A0
:1018D000CE13D8F9FFE9121DA8EFF0121CCFCEC32A
:1018E00013CE13D8F9121DBB2445F582E434FFF55D
:1018F00083EFF0E9121DCEE975F008A42446F582C5
:10190000E434FFF5837480F00219677878E6540FA9
:10191000F9121D9A121DB62407F582E434FF121C39
:10192000C8CEC313CE13D8F9121DBB2401F582E42F
:1019300034FFF583EFF0121CCFCEC313CE13D8F9CA
:10194000121DBB2405F582E434FFF583EFF0E97541
:10195000F008A42402F582E434FFF583E4F0E9758D
:10196000F008A42406F582E434FFF583E4F00523AF
:10197000E52364046003021891903209E493FF7830
:1019800078F6121D98E4F090320893FFF6121D4588
:10199000E4F090FFFD7405F0227B007A007923903B
:1019A000FACFE475F001121B3285F02EF52D7D0182
:1019B000022698E709F608DFFA8046E709F208DF11
:1019C000FA803E88828C83E709F0A3DFFA8032E355
:1019D00009F608DFFA8078E309F208DFFA807088F8
:1019E000828C83E309F0A3DFFA806489828A83E032
:1019F000A3F608DFFA805889828A83E0A3F208DF21
:101A0000FA804C80D280FA80C680D4806980F280CF
:101A100033801080A680EA809A80A880DA80E280F5
:101A2000CA803389828A83ECFAE493A3C8C582C84A
:101A3000CCC583CCF0A3C8C582C8CCC583CCDFE9B4
:101A4000DEE7800D89828A83E493A3F608DFF9EC50
:101A5000FAA9F0EDFB2289828A83ECFAE0A3C8C5DB
:101A600082C8CCC583CCF0A3C8C582C8CCC583CC02
:101A7000DFEADEE880DB89828A83E493A3F208DF71
:101A8000F980CC88F0EF60010E4E60C388F0ED2441
:101A900002B4040050B9F582EB2402B4040050AF44
:101AA00023234582239019FC73BB010689828A8314
:101AB000E0225002E722BBFE02E32289828A83E40D
:101AC0009322BB010CE58229F582E5833AF583E098
:101AD000225006E92582F8E622BBFE06E92582F8B7
:101AE000E222E58229F582E5833AF583E49322BB7D
:101AF000010689828A83F0225002F722BBFE01F39D
:101B000022F8BB010DE58229F582E5833AF583E8E9
:101B1000F0225006E92582C8F622BBFE05E925829F
:101B2000C8F222C5F0F8A3E028F0C5F0F8E5821568
:101B30008270021583E038F022A3F8E0C5F025F0AA
:101B4000F0E582158270021583E0C838F0E822BB08
:101B50000110E58229F582E5833AF583E0F5F0A3EB
:101B6000E0225009E92582F886F008E622BBFE0A49
:101B7000E92582F8E2F5F008E222E5832AF583E917
:101B800093F5F0A3E99322BB010A89828A83F0E5E9
:101B9000F0A3F0225006F709A7F01922BBFE06F3C6
:101BA000E5F009F31922F8BB0111E58229F582E578
:101BB000833AF583E8F0E5F0A3F0225009E92582A5
:101BC000C8F608A6F022BBFE09E92582C8F2E5F0B6
:101BD00008F222A42582F582E5F03583F58322E61A
:101BE000FB08E6FA08E6F922EBF608EAF608E9F659
:101BF00022E0FBA3E0FAA3E0F922EBF0A3EAF0A3D2
:101C0000E9F022D083D082F8E493701274019370CB
:101C10000DA3A393F8740193F5828883E47374028F
:101C2000936860EFA3A3A380DFAB36AA37A938E59A
:101C30004C121AE874012538F538E43537F537AB1E
:101C400036FAA9387411121AE874012538F538E407
:101C50003537F53790FF06E0AB36AA37A938121AA8
:101C6000E874012538F538E43537F537AB36FAA98D
:101C700038E4121AE8042538F538E43537F537AB7F
:101C800036FAA938E4121AE8042538F538E435376D
:101C9000F53790FF04E0AB36AA37A938121AE8747A
:101CA000012538F538E43537F53790FF05E0AB36D8
:101CB000AA37A938121AE874012538F538E43537FF
:101CC000F53722F583E05408AB36AA37A93822F558
:101CD00083EFF0FD7C00C3787BE69DF618E69CF66A
:101CE000E6FE08E67803227536017537F975387215
:101CF00022E04404F074132FF582E434F9F583E014
:101D00002290FABCE0FF7E00C390FAC0E09FF09002
:101D1000FABFE09EF090FAB7EE8FF0121B1CEF2591
:101D20004FF54FEE354EF54E227B017AFA79B4909D
:101D3000FAB7E0F52DA3E0F52E22787CE6FE08E662
:101D40008E832404F582E43583F58322540F75F0E5
:101D500008A42440F582E434FFF58322E54D75F0B4
:101D600008A42448F582E434FF22E54D75F008A468
:101D70002408F582E434FF2290FAB9E0FF24FC2223
:101D800090FF00E0541F2290FABEE090FABAF022D1
:101D90007533008F3490F96F121BEA9000022254C1
:101DA0000F75F008A42400F582E434FFF583227552
:101DB000F008A42441F582E434FFF583227480F016
:101DC00008E6FFE975F008A42274B22522F582E442
:101DD00034FAF5832275F008A42442F582E434FF36
:101DE000F5837480F02290FF82E04408F02290FF97
:101DF000FEE04403F090FFFCE054FDF0227867E63B
:101E000054FDF690FFFD7465F022121BCCE0FEA39A
:101E1000E0FF4E227B017AFA79B72290FF80E044FE
:101E200008F02290FF83E0547FF022E0FF90F96AEF
:101E3000021BEA90FFA4E04402F022753901753AD2
:101E400009227B017AF9797222D3E53C9408E53BBB
:101E500094012290FABEE0FF90FABAF02290FFA41B
:101E6000E054EF2290FFB4E054EF2212104B788838
:101E7000EFF6122AC71222FA8E8324091222A1E059
:101E8000FD1222E890000A122302240A1222A1E085
:101E900090000B121AFA1222FAF5828E83A3A3A3E2
:101EA000E0F55312230624041222A1E0F5548F8298
:101EB0008E83A3A3E0F555E553C41313135401789F
:101EC00088F6D394004006E55430E101067888E6B0
:101ED0001222E790000CEF121AFA1222B5A3A3E027
:101EE000FEA3E0FF53070C5306E6E55330E503433A
:101EF0000701E55420E50EE553547F7008E55320B3
:101F0000E703430702E55330E303430710E553308B
:101F1000E203430720E55354036003430740E553BE
:101F200030E103430780E55330E403430601E55302
:101F300030E603430608E55420E40EE553547F7071
:101F400008E55320E7034306105307FB5306799037
:101F50000005EE8FF0121B9FE55530E3125430FF61
:101F6000C4540F1222E7900008EF121AFA800A12E6
:101F700022E8900008E4121AFAE55554031222E709
:101F8000900007EF121AFAE5555404FFC3139000AE
:101F900009121AFA900007121ABB70131222E8E90C
:101FA0002409F9E43AFA121AA2FFC313121AE8122A
:101FB000232724081222A1E0FE8D828C83E582244F
:101FC000071222A1E0FDEEED1222E7900003EE8F52
:101FD000F0121B9F1232847D0AE4FF122FB402100C
:101FE000CE90FAE6E0B403067E007F4080047E00D7
:101FF0007F0890FADAEEF0A3EFF0900005121ABB1A
:10200000FF7E0090FAD6EEF0A3EFF070037F082277
:10201000900008121B48FF90FAD8E5F0F0A3EFF00B
:10202000AE02AF018E508F51740A2551F551E4353F
:1020300050F55090FADBE0FF14FE90FAD9E05EFE16
:10204000C3EF9EFF90FADDF0C390FAD7E09F90FABD
:10205000D6E094005006A3E090FADDF01220A960CB
:1020600003E0FF22122E2B90FAD6E0FEA3E0FF4EF3
:10207000602B90FADAE0FCA3E0FDD3EF9DEE9C40EC
:1020800007E090FADDF0800890FAD7E090FADDF0F2
:102090001220A96003E0FF22122E2B80CA7B007A57
:1020A000007952E4F52DF52E7D011226987F00224D
:1020B000AA50A9517B0190FAD8E0FCA3E0FD90FA68
:1020C000DDE0F54A12296090FADCEFF022EF24AE51
:1020D000605224FE602E24FE7003022169240660F3
:1020E000030221B17871E654FBF690FFA5E0F522DA
:1020F000440FF0743390FA94F0E522A3F090FAB212
:102100007401F0227872E654FBF690FFB5E0F522F8
:10211000440FF0744390FA96F0E522A3F090FAB3DE
:102120007401F02290FAA0E0A320E5030221B1900F
:10213000FFA6E090FACDF0A3F090FACDE0FF540FA7
:10214000FE601090FFA612230D90FFA6E090FACD3E
:10215000F080E690FACEE0FF7434FE122D85EF7029
:102160005790FACEE0FF743490FA98F0EFA3F02283
:1021700090FAAAE0A330E54090FFB6E090FACDF0E7
:10218000A3F090FACDE0FF540FFE601090FFB6125E
:10219000230D90FFB6E090FACDF080E690FACEE005
:1021A000FF7444FE122D85EF700E90FACEE0FF749E
:1021B0004490FA9AF0EFA3F022C0E0C0F0C083C0D0
:1021C00082C0D075D000C000C001C002C003C004EE
:1021D000C005C006C00790FF92E0FF90FACCF090D7
:1021E000FF92E4F0EF121BFC22692622692E220CDA
:1021F00030220C32221A38222C3A225E3E224944E6
:10220000223E462254502254522254542254560004
:1022100000226E90FACCE0FD7C007F0112115E80FE
:10222000627C007D017F0312115E90FFFEE044207E
:10223000F080507C007D017F0212115E90FFFEE075
:102240004440F0803E7C007D017F0512115E8033AA
:102250007C007D017F0612115E802890FACCE0FFA1
:102260001220C6801E7C007D017F0412115E801347
:1022700012284E800E90FACCE02400FFE434FFFEDA
:10228000122D85D007D006D005D004D003D002D0BF
:1022900001D000D0D0D082D083D0F0D0E032787C92
:1022A000E6FE08E624048E83F582E43583F5832276
:1022B00074132524F582E434F9F583227880E6FE50
:1022C00008E6F5828E83227880E6FE08E6AA06F804
:1022D000AC027D017BFF7A3279567E007F0A021ABA
:1022E0007C7880E6FC08E6F5828C83A3A322FF902D
:1022F000F96F021BEA90F96A121BEA900004021AB5
:10230000BB787EE6FE08E6FF22ED121AFA8F828E77
:1023100083E58222EFF090FACEE0540F4EFEF0EF0C
:1023200054F04EF0227880E6FC08E68C8322787E1A
:10233000E6FC08E6FD8C8322A607E6246EF8E6227A
:10234000787EE6FA08E6FB2208E6FE08E68E83229F
:1023500026F618EE36F622EF240BF582E43EF583DE
:10236000228B828A83E582228B258A2689278D28E3
:1023700090FAD2E4F0A37402F07B017AFA79D1905A
:10238000FAD2E0F52DA3E0F52E7D0112269890FA01
:10239000D1E065286046A3E0FFA3E0A3CFF0A3EF60
:1023A000F01223F090FAD1E0FF90FAD4E48FF0120B
:1023B0001B1C1223F090FAD4E0FFA3E090FAD2CFD6
:1023C000F0A3EFF090FAD1E0A375F000121B1C907F
:1023D000FAD2E475F004121B1C02237290FAD3E0C7
:1023E0002401FF90FAD2E03400AB25AA26A9278F5A
:1023F000F0121B807F00227B017AFA79D190FAD209
:10240000E475F001121B1C85F02EF52D7D010226CE
:10241000988F62122AC71222FA8E83240B1222A1ED
:10242000E054FBF04402F0081222DCE0A330E50C9B
:10243000122306240B1222A1E04401F0787CE6FE70
:1024400008E6FFF5828E83E054B8FDF0E56224FED5
:102450004420FC4DF0E58224041222A1E054B8F09F
:102460004CF08F828E83A37403F018E6FE08E6FF1B
:102470008E8324051222A1C083C082E0FD749925B9
:1024800062F582E434FAF583E054FC4403FCED4C3D
:10249000D082D083F08F828E83E04480F0E5822466
:1024A000041222A1E04480F0123284746E2562F896
:1024B000740446F67F002212104B7F0212126178DC
:1024C00067E64402F6D2B0D2B190F916E030E707E1
:1024D00090FF9EE4F08036D2B390FFA4E090FA7EA5
:1024E000F090FFB4E090FA7FF090FFA2E090FA7CC9
:1024F000F090FFB2E090FA7DF090FFA47430F0907D
:10250000FFB4F090FFA27440F090FFB2F090FAE7B1
:10251000E5A8F075A88190FF92E06004E4F080F6F1
:1025200090FFFD743AF043870100000090FA7EE0CE
:1025300090FFA4F090FA7FE090FFB4F090FA7CE076
:1025400090FFA2F090FA7DE090FFB2F090F918E0D1
:102550006002C2B390FAE7E0F5A80210CE8B5C8A65
:102560005D895E122E0D90FAC3121BF3AA5DA95E5F
:1025700090FAC6121BF390FAC7E475F00A121B1CFE
:1025800090FAC6121BEAE92401F9E43AFA90FAC972
:10259000121BF3AB5CAA5DA95E122E19E0FFC313F8
:1025A000F0E47882F690FAC1E0FF7882E6C39F50AB
:1025B0004A90FAC3122DEEFF7883F690FAC6122DD8
:1025C000EEFEF45FFF7883F6122DEB5E4FFF78830B
:1025D000F6122DF475F002121B1C90FAC7E475F088
:1025E00002121B1CAB5CAA5DA95E900004121ABB10
:1025F00030E403122E0378820680AAE490FAC2F037
:10260000228B568A57895890FAC27406F0E490FAE1
:10261000C1F0121AA2246E6026147070122DDA60B6
:1026200009243070121225568062122E24121FDAED
:1026300090FAC2EFF0805590FAC27481F0804D128A
:102640002DDA60092430703E122D30803FE5582489
:1026500003F9E43557FA7B01C003C002C001122E12
:1026600024900005121ABBFD900008121B48F52E9D
:1026700085F02DD001D002D00312269890FAC1EF38
:10268000F0E4A3F0800690FAC27481F090FAC2E000
:10269000122E24900002121AFA90FAC1E0FF228B47
:1026A000298A2A892B8D2CE52C7003AF2C22122E1F
:1026B000537016122E72E52D90FFF1F01231D850A2
:1026C000F2122725400B7F0022122E72122725506E
:1026D000F890FFF374A1F0E52CB4010790FFF0E04F
:1026E0004402F090FFF1E4F0F52FE52C14FFE52F04
:1026F000C39F502A1231C14003AF2F22C3E52C954E
:102700002FFFBF020790FFF0E04402F0122E650594
:102710002F7401252BF52BE4352AF52A80CC1231B4
:10272000C140037F1822122E65AF2C2290FFF1E5E5
:102730002EF00231D812104B788412233130E10888
:102740007F131231A90227BC7884E6F924131222E0
:10275000ADE0FF30E7405403601EE9B4030D90FF85
:102760009EE054FEF0E04404F0804690FF9EE0546A
:10277000FDF0E04408F08039E9B4030D90FF9EE0DD
:1027800054FBF0E04401F0802890FF9EE054F7F005
:10279000E04402F0801BEF54036014E9B403099095
:1027A000FFA4E054DFF0800790FFB4E054DFF0C2F4
:1027B000B390F918E004F0AF011222EEFD122FE5FC
:1027C0001231A90210CE75A840787FE4F6D8FD75C5
:1027D000818B02280902318CE493A3F8E493A3408F
:1027E00003F68001F208DFF48029E493A3F854078C
:1027F000240CC8C333C4540F4420C8834004F45687
:10280000800146F6DFE4800B0102040810204080BE
:10281000902BA9E47E019360BCA3FF543F30E509EF
:10282000541FFEE493A360010ECF54C025E060A8BE
:1028300040B8E493A3FAE493A3F8E493A3C8C58251
:10284000C8CAC583CAF0A3C8C582C8CAC583CADFBF
:10285000E9DEE780BEE4F522121DC2E0B4040DE516
:10286000222403FF123013121DC2E4F00522E522D8
:10287000C3940240E3E4F52275F002E52290FA9455
:10288000121E03602C122D85EF605275F002E522B6
:1028900090FA94121BCCE4F0A3F075F00AE52290B4
:1028A000FAA0121BCCE0A330E633121DC27404F070
:1028B0002275F002E52290FA98121E036016122D7E
:1028C00085EF601975F002E52290FA98121BCCE4AE
:1028D000F0A3F0220522E522C39402409B22E4FFEC
:1028E00090FF83E0540FFEEFC39E501774F02FF556
:1028F00082E434FEF583E0121CC1121AE80F121CA8
:10290000B080DDEFFDC3E53A9DF53AE5399400F579
:1029100039D3E53A9400E53994004006E490FF830A
:10292000F022121DDF121E34121E26121AA2246E6D
:10293000601E14601B248E702D900001121ABBFFC4
:1029400024FC600304701FEFFD7C007F0D02115E0C
:10295000121E3B1225FA121D89121ABB60030232A5
:102960007AE4FF12326E228B458A4689478C488D65
:1029700049D200122E537016122E72E54890FFF1C4
:10298000F01231D850F21229D5400B7F1822122EA6
:10299000721229D550F8E4F54BE54A14FFE54BC314
:1029A0009F50171229C540037F1822054B7401253B
:1029B00047F547E43546F54680DF90FFF0E04401F7
:1029C000F01229C540037F18227F0022AB45AA469A
:1029D000A947121AA290FFF1F00231D890FFF1E559
:1029E00049F00231D87B017AFA79CFE4FD122361F4
:1029F00090FACFE475F009121B1C7B007A00792352
:102A000090FACFE475F001121B3285F02EF52D7D82
:102A10000112269890FFF7E523122A3990FFF6E578
:102A200023F090FACFE4F0A37406122A39E523309C
:102A3000E00790FFFC7494F02290FFFC7490F02269
:102A4000F07B007A00792390FACFE475F001121B35
:102A50003285F02EF52D7D0102269890FF9374812A
:102A6000F090FFFFE0600690FFFC7410F090FF9183
:102A7000E04490F0E490F916F0A3F0122B3912160E
:102A8000C91230697E077FD012122A7E0F7FA012F2
:102A90001244E47877F67877E6FFC39406500B7417
:102AA0006E2FF8E4F678770680EC7F031230B29050
:102AB000F916E020E4057F041230B290FF9BE4F0A9
:102AC00090FF9AF090FFE8E0541FF0D2A82215651D
:102AD000A865A6073008051211AE80F8D208A865CF
:102AE000E6FFB4030F787C76FF0876E00876FF08EF
:102AF00076A0800D787C76FF0876E20876FF08766F
:102B0000B0788076FA08769EEF24FD75F00AA4AEC0
:102B1000F01223497B017AFF79487868121BE1A8FB
:102B200065E624FD75F008A4FFAEF0786A1223492B
:102B30007908786B121BE1786DEF12234905652245
:102B400090FFF0E054ABF0E04420F090FAE674021D
:102B5000F07B017AFA79CFE4F52DF52E7D0112266E
:102B6000987E0090FAE4EEF0A3EFF064017010900C
:102B7000FACFE0B4520990F916E054EFF0802990B2
:102B8000FAE4E07004A3E06401701090FACFE0B4BE
:102B9000100990F916E04410F0800D90FAE67403E5
:102BA000F090F916E054EFF090FFF0E04420F022AE
:102BB000036801FF48036B01FF080266000044FA46
:102BC000980000000044FA940000000042FAB200AD
:102BD0000042FA7E000042FA7C000042F96DFFFFDD
:102BE00042FA7A000041F966FF41F91C1941F915D2
:102BF0000043F9190A320241F9682041F96920417C
:102C0000F9650041F9670044F8000000000042F94E
:102C100016000041F9180001200041F804000012DC
:102C2000104B788AEFF6122AC71222EE30E029788C
:102C30007C1222B7E0547FF0786B121BD890000210
:102C4000121ABB30E709900002E4121AFA80E97800
:102C50007C1222B7E04480F01222EE30E11E1222F4
:102C600097E0547FF01232197868121BD890000256
:102C70007480121AFA122297E04480F0123284E42F
:102C8000FF1231A90210CE12104B7885EFF61231E7
:102C9000501231A97885E6FF24131222ADE0FE30F0
:102CA000E716EFB4030990FF9EE054FAF0802290FB
:102CB000FF9EE054F5F08019EE54036014EFB40366
:102CC0000990FFA4E04420F0800790FFB4E0442086
:102CD000F090F918E014F0E07002D2B30210CE12B6
:102CE0001E1CE53A64097004E53964016048C3E5D7
:102CF0003A9408E539940040117F08EFE53A9408CA
:102D0000F53AE5399400F5398005AF3A121E34E4FE
:102D1000FEEEC39F5019121CC1121AA2FD74F82EA8
:102D2000F582E434FEF583EDF00E121CB080E2EF84
:102D3000547F90FF81F0228B598A5A895B122E1999
:102D40007005A37408F022AB59AA5AA95B122E0D84
:102D500090FAC9121BF3E55B2403F9E4355AFA90A3
:102D6000FAC3121BF3E490FAC2F0788BF690FAC122
:102D7000E0FF788BE6C39F5012122DEBFF122DF46B
:102D8000122E07788B06122E0380E222AD07AC06C6
:102D900090320AE493FF7874F6540F121DA8E008ED
:102DA000760008F618121CD9C333CE33CED8F9FFFB
:102DB0007875EEF608EFF6EE44F818F6EF08F690A0
:102DC000FF7AE020E7037F00227875E6FE08E6F54B
:102DD000828E83ECF0A3EDF090FF7A7402F07F0115
:102DE00022AB56AA57A958900003121ABB54F024DC
:102DF000A02290FAC9121BEA021AA290FAC3121B6F
:102E0000EAEF121AE890FACAE42290FAC4E475F0E4
:102E100001021B1C900008121B48AAF0F97B01223A
:102E2000900005121ABB90FAC1F022AB56AA57A91E
:102E3000582290FADDE0FF7E00C390FAD7E09FF0C1
:102E400090FAD6E09EF090FAD8EE8FF0121B1CEFAD
:102E50002551F551EE3550F5502290FFF0E054FE2B
:102E6000F0E054FDF090FAE6E064032290FFF2E017
:102E7000AB29AA2AA92B021AE890FFF374A0F0222A
:102E80008F64ED700FE564B403057F010231EF7FBD
:102E9000020231EFAF64122AC7746E2564F8E6307F
:102EA000E20BD209121D33E0547FF08002C209E523
:102EB00064B403077F811231EF80057F821231EF06
:102EC000300907121D33E04480F0123284221210C0
:102ED0004B90FFFDE04460F0D20190FFFCE0440223
:102EE000F090FF00E030E71390FF83E04480F04370
:102EF000358090FFFCE04401F0800D121DDF53355A
:102F00007F90FFFCE054FEF090FF81E04480F012DF
:102F100002DE121DE70210CE12104B7889EFF6D2B6
:102F200000122AC790F96A121BEAE92403F9E43A6D
:102F3000FAC0027880E6FE08E6AA06F8AC027D0137
:102F4000D0021222D31232847889E6FF121387123C
:102F500031A90210CE8F63122AC7787C1222B7E003
:102F6000543FF0E58224041222A1E0543FF01223E2
:102F700041240B1222A1E054F8F0123284746E2521
:102F800063F874FB56F67F002212104B122AC71208
:102F900022FA240612229FE0FD1222E8900003127A
:102FA000230224051222A1E0900004121AFA123220
:102FB000847D02E4FF122FB40210CEAE05121D8EE6
:102FC000EF121AFA0E0E0EEED3953CE4953B40023A
:102FD000AE3CEED3940874809481400A7E03900046
:102FE000027402121AFAAF0612326E22AE07ED54C4
:102FF00003640160037F1022ED547CC394045003EA
:103000007F0B22746E2EF8740246F674992EF582A8
:10301000E434FAF583EDF07F0022BF03067CFF7DE8
:10302000E080047CFF7DE28D828C83E04480F0E5CB
:103030008224041222A1E04480F0746E2FF87404FC
:1030400046F67F002212104BE53A64097004E53918
:103050006401601690FF83E0540FFFC3E53A9FE5DB
:1030600039940040051228D7800312327A0210CE1C
:1030700090FFFCE020E71FC2AF7DFFAC051DEC60B8
:10308000157E047F00EF1FAA0670011E4A60EC90B7
:10309000FF92E4F080EF2212104B7866E6FE08E61D
:1030A000FF30E01230E10F90FFFCE04420F07F049D
:1030B000121261121DF60210CE8F23C208122AC707
:1030C0001222C0787E122342240B1222A1E054F86F
:1030D000F0123284AF23121387228E5F8F60E56077
:1030E0001560AE5F7002155FD39400EE9400400946
:1030F0007E077FD012102480E52211DC2EC724B079
:1031000032603090303E316F2F82272E2C8031126A
:1031100031311E642F112C180E12104B7886122399
:103120003120E1077F121231A9800A7886E6FF126A
:10313000240A1231A90210CE12104B7887122331C3
:1031400020E2077F111231A9800A7887E6FF122F4B
:103150004E1231A90210CE8F61122F4EAF61122A8A
:10316000C71222C0123284746E2561F874FD56F6BF
:10317000AF611213872212104BE53A64097004E51F
:103180003964016005122CD88006121E14121E1C10
:103190000210CE122A5412130390F804E0FF6005C7
:1031A0007D011212A01229DE12133F1211BC80E31E
:1031B000121D8EEF121AFAE4F533F534EF600302B4
:1031C000327AE4FF12326E2290FFF0E0FF54A060EA
:1031D000F7EF30E50890FFF04420F0C322D32290AF
:1031E000FFF0E0FF542860F7EF30E50890FFF0446F
:1031F00020F0C322D322EF30E708121D45E054DF50
:10320000F022EF121D98E054DFF022810182028348
:10321000038740004000400040004000400008009C
:10322000787E1222B7A3A3E0FF30E706547FF04474
:1032300080F022853B39853C3A90FF82E054F7F0DC
:10324000A3E0547FF022E4FEEE90320493B507022F
:10325000D3220EBE07F2C32200081828380181903D
:103260000A02000011130012104B7F021210DA1232
:103270001DF60210CE7539008F3A121CE0122CD8C0
:0E32800022121E1C121DDF121E1422C2082272
:00000001FF
